:020000040000FA
:0600000097EF2CF0120046
:0600080004EF08F01200F5
:060018000CEF08F01200DD
:0610000097EF2CF0120036
:061008001CEF08F01200CD
:061018006FEF09F0120069
:06102A00010090590000D6
:0810300000020000A200000014
:08103800DACFE4FFE2CFDAFF9A
:10104000E9CFE4FFEACFE4FFF6CFE4FFF7CFE4FF18
:10105000F5CFE4FFF3CFE4FFF4CFE4FFFACFE4FFF2
:1010600000EE00F0140EE80403E3EECFE4FFFBD73C
:1010700000EE14F00C0EE80403E3EECFE4FFFBD720
:10108000E65220EC20F0F2A406D101019B2B000EC9
:101090009C2302010F51101101E1EDD013071351F0
:1010A00001E0E9D016C220F0216A226A20AE02D007
:1010B00021682268205081272150822322508323D7
:1010C000A3C113F29F5102E1A3C113F2F00E8114E8
:1010D0000101A26F02011651255D4EE016C220F0FB
:1010E000216A20BE216820501D2721501E23205137
:1010F0001E19E8AE02D01E3504D01D511F5D1E51D1
:10110000205904E221C21DF222C21EF21E512219F0
:10111000E8AE02D0223504D021511D5D22511E5966
:1011200004E21FC21DF220C21EF216C220F0216A84
:1011300020BE216820501D2721501E2320511E193A
:10114000E8AE02D01E3504D01D511F5D1E5120593E
:1011500004E221C21DF222C21EF21E512219E8AE83
:1011600002D0223504D021511D5D22511E5904E2C6
:101170001FC21DF220C21EF216C225F2270E1D2527
:10118000E96E020E1E21EA6EEF500101A213A2C108
:1011900081FF16C220F0216A20BE21682050020182
:1011A0001D2721501E2320511E19E8AE02D01E35E6
:1011B00004D01D511F5D1E51205904E221C21DF2B1
:1011C00022C21EF21E512219E8AE02D0223504D0EE
:1011D00021511D5D22511E5904E21FC21DF220C281
:1011E0001EF20F07000E105B0F51101144E1136B3C
:1011F000A6840A0EA96E100E1F0B81C220F082C2B7
:1012000021F083C222F006E0D8902232213220322F
:10121000E806FAE1216A226A2050A86EB0EC1AF0C2
:10122000A6840B0EA96E080E1F0B81C220F082C28D
:1012300021F083C222F006E0D890223221322032FF
:10124000E806FAE1216A226A2050A86EB0EC1AF092
:10125000A6840C0EA96E81C220F0216A226A205059
:10126000A86EB0EC1AF005C2AAF106C2ABF10201F9
:10127000995101E0996B13510F11206E10C221F0AA
:10128000E850211007E1245105E0F00E811401011E
:10129000A26F816EF294E55200EE1FF00C0EE8048E
:1012A00003E3E5CFEDFFFBD700EE13F0140EE804E7
:1012B00003E3E5CFEDFFFBD7E5CFFAFFE5CFF4FF82
:1012C000E5CFF3FFE5CFF5FFE5CFF7FFE5CFF6FF7D
:1012D000E5CFEAFFE5CFE9FFE5CFDAFF1100D8CF90
:1012E000E4FFE0CFE4FFE46EDACFE4FFE652E5523C
:1012F000E5CFDAFFE550E5CFE0FFE5CFD8FF1000FE
:1013000093908A9093948A92816A7CDA08EC28F010
:1013100093909392939493968A92F19EF00E8114F7
:101320000101A26F816E0201136B146B196B1A6BB2
:10133000F28AF294F184D59ED58CD59AD596D5842F
:10134000D592D590D768D66A0F6B106BFF0E0F5DE4
:101350007F0E105905E2A69E0F2B000E1023F6D724
:101360000F6B106B230EA96EA69EA69CA680A8CF1D
:10137000A3F1A3C1A5F1A69E010EA96EA680A8CFD8
:10138000A4F1A69E020EA96EA680A8CF1BF2A69E6F
:10139000030EA96EA680A8CF24F2A69E040EA96E05
:1013A000A680A8CF26F2A69E0A0EA96EA680A8CF78
:1013B00084F2856B866B100E1F0B84C281F285C28E
:1013C00082F286C283F207E00201D8908137823729
:1013D0008337E806FAE1A69E0B0EA96EA680A8CF79
:1013E00084F20201856B866B080E1F0B84C214F019
:1013F00085C215F086C216F006E0D8901436153670
:101400001636E806FAE114500201812715508223AE
:1014100016508323A69E0C0EA96EA680A850146EAB
:10142000156A166AE85081131550821316508313FB
:10143000A69E0F0EA96EA680A8CFA9F1A69E0E0E9D
:10144000A96EA680A8CFA7F1A69E050EA96EA680BC
:10145000A8CFB2F1A69E060EA96EA680A8CFB0F1C5
:10146000A69E1F0EA96EA680A8CF03F20101040E4E
:10147000906F1E0E8F6F8F510D0873E2A69E020EA5
:101480008F5DA96EA680A8CF84F20201856B866B62
:10149000100E1F0B84C214F085C215F086C216F020
:1014A00006E0D890143615361636E806FAE1010142
:1014B0009051030DF3CFE9FFF4CFEAFF8A0EE9263E
:1014C000020EEA2214C0EEFF15C0EEFF16C0EEFFBA
:1014D000A69E8F05A96EA680A8CF84F20201856B17
:1014E000866B080E1F0B84C214F085C215F086C2ED
:1014F00016F006E0D890143615361636E806FAE1EE
:1015000001019051030DF3CFE9FFF4CFEAFF8A0EFA
:10151000E926020EEA221450EE261550EE2216504D
:10152000EE22A69E8FC1A9FFA680A8CF84F2020159
:10153000856B866B01019051030DF3CFE9FFF4CF6A
:10154000EAFF8A0EE926020EEA2202018451EE1217
:101550008551EE128651EE1201019007030E8F5F46
:101560008AD7550EA35D06E1A69EA96AA680A8CFDC
:10157000A3F1F3D0550EA36FA69EA69CA684230EBE
:10158000A96EA3C1A8FFA5EC1AF00101140EA36F68
:10159000A69EA69CA684A96AA86EA5EC1AF00101D5
:1015A0000F0EA46FA69EA69CA684010EA96EA4C1D0
:1015B000A8FFA5EC1AF002010A0E1B6FA69EA69CBE
:1015C000A684020EA96E1BC2A8FFA5EC1AF00201A8
:1015D000246BA69EA69CA684030EA96E24C2A8FF17
:1015E000A5EC1AF00201266BA69EA69CA684040E0A
:1015F000A96E26C2A8FFA5EC1AF00201816B826BCE
:10160000836BA69EA69CA6840A0EA96E100E1F0BC5
:1016100081C214F082C215F083C216F006E0D890A1
:10162000163215321432E806FAE1156A166A1450B9
:10163000A86EA5EC1AF0A69EA69CA6840B0EA96E19
:10164000080E1F0B81C214F082C215F083C216F07F
:1016500006E0D890163215321432E806FAE1156A1F
:10166000166A1450A86EA5EC1AF0A69EA69CA68435
:101670000C0EA96E81C214F082C215F083C216F05E
:10168000156A166A1450A86EA5EC1AF00101A96B30
:10169000A69EA69CA6840F0EA96EA9C1A8FFA5ECC4
:1016A0001AF0A69EA69C0101A76BA6840E0EA96E39
:1016B000A7C1A8FFA5EC1AF0A69EA69C0101B26BDB
:1016C000A684050EA96EB2C1A8FFA5EC1AF0A69ECD
:1016D000A69C0101B06BA684060EA96EB0C1A8FF3E
:1016E000A5EC1AF0A69EA69C0201010E036FA6842B
:1016F0001F0EA96E03C2A8FFA5EC1AF00101040E8B
:10170000906F1E0E8F6F8F510D0827E29051030DC1
:10171000F3CFE9FFF4CFEAFF8A0EE926020EEA22B0
:10172000EE6AEE6AEE6AA6848FC1A9FFA86AA5ECEC
:101730001AF0A68401018F05A96EA86AA5EC1AF01B
:10174000A684020E01018F5DA96EA86AA5EC1AF0AD
:1017500001019007030E8F5FD6D7D58E02011C6B57
:10176000030E2603F3501525E96EEA6AD890E93690
:10177000EA366F0EE926020EEA22EFCF21F2226B43
:1017800021BF2269030E2603F3501525E96EEA6A8C
:10179000D890E936EA366F0EE926020EEA22010EEB
:1017A000E926000EEA22EFCF1FF2206B1FBF20694F
:1017B000136B21C21DF222C21EF2E6D8020E0201F4
:1017C0009F5D02E186EC1CF002019F05F6E19E514F
:1017D00013E00F511011F1E19E6BF29E0101B25125
:1017E0009D2502010F6F000E01019E210201106F65
:1017F000B1C116F2F28EE1D70F511011DEE19D6BEF
:101800009F6BDBD70F0EC11202D8B4EF1FF0D9CFF8
:10181000E6FFE1CFD9FFE6521FD8DF6ADF50146E32
:10182000156A400E145C000E155809E2DF50EA6A92
:10183000000FE96E010EEA22EF6ADF2AEFD70101FD
:10184000806B816B836B846BC00E89169216E55298
:10185000E552E7CFD9FF1200D9CFE6FFE1CFD9FF9C
:10186000E652948E949C240EAC6E900EAB6EE20EFB
:10187000AF6E040EB06E080EB86EAE50DF6EE5525D
:10188000E552E7CFD9FF1200D9CFE6FFE1CFD9FF6C
:10189000ACA2FED7FE0EDB50AD6EE552E7CFD9FF0E
:1018A0001200D9CFE6FFE1CFD9FFACA2FED7FE0EE2
:1018B000DB50AD6EE552E7CFD9FF1200D9CFE6FF7E
:1018C000E1CFD9FF040EE126D880000E05010055B6
:1018D000C20E0155010E0255000E035537E300C537
:1018E00088F501C589F502C58AF503C58BF5186A27
:1018F0001B0E196EB70E1A6E1B6A18C006F019C0BF
:1019000007F0086E1BC009F088C50BF089C50CF004
:101910008AC50DF08BC50EF009EC2CF006C014F052
:1019200007C015F008C016F009C017F01406000E25
:10193000155A165A175A14C0DFFF010E15C0DBFFE7
:10194000020E16C0DBFF030E17C0DBFF040EE15CC6
:1019500002E2E16AE552E16EE552E7CFD9FF1200FB
:10196000D9CFE6FFE1CFD9FFE652ABA205D0AB98C5
:10197000AE50DF6EAB8802D0AE50DF6EDF50E55266
:10198000E552E7CFD9FF1200D9CFE6FFE1CFD9FF6B
:10199000E652F8EC19F08BEC1DF0200E0101E76E19
:1019A000B519E8AE02D0E73402D0E750B55D03E3E5
:1019B0006D50020B02E029EF16F00201005116E112
:1019C000400EE66E400EE66E010EE66EA3EC28F0C9
:1019D000E552E552E5520101816F01018151000894
:1019E00005E20201010E006F0101826B020100514C
:1019F00002E113EF16F001018251EA6A400FE96E2D
:101A0000010EEA22EFCF85F102010251090A02E13B
:101A100086EF14F00C0A02E164EF14F0010A02E10F
:101A200035EF14F0070A02E118EF14F0110A02E191
:101A3000F9EF13F0100A02E1DCEF13F0150A02E1EE
:101A4000B7EF13F00F0A02E160EF13F0070A02E1AB
:101A5000B1EF12F03F0A02E1B1EF12F0010A02E128
:101A6000B1EF12F0030A02E1B1EF12F0010A02E154
:101A7000B1EF12F0070A02E1B1EF12F0010A02E140
:101A8000B1EF12F03B0A02E190EF12F0530A02E1CB
:101A90001DEF12F05E0A02E1D3EF11F05F0A02E1DE
:101AA000A2EF11F0580A01E1F2D21B0A01E1EBD2D8
:101AB000010A01E1D6D21F0A01E1CCD2010A01E1FB
:101AC000B1D2060A01E18BD25F0A01E16DD2030AAD
:101AD00001E106D2010A01E1B1D14A0A01E16AD16C
:101AE000140A01E126D15B0A01E17DD04E0A02E031
:101AF00007EF16F0060E0101855D18E102011C6B6F
:101B000001018051EA6A000FE96E010EEA22530ECC
:101B1000EF6E0101802B01018051EA6A000FE96E2E
:101B2000010EEA22EF6A0AEF16F056D0530E0101B9
:101B3000855D32E102011C6B02010F51101116E0AC
:101B400001018051EA6A000FE96E010EEA22310EAE
:101B5000EF6E0101802B01018051EA6A000FE96EEE
:101B6000010EEA22EF6A0AEF16F015D0010180514A
:101B7000EA6A000FE96E010EEA22300EEF6E0101F3
:101B8000802B01018051EA6A000FE96E010EEA2202
:101B9000EF6A0AEF16F020D0510E0101855D08E1D1
:101BA00002011C2B0201150E026F0AEF16F014D071
:101BB000500E0101855D08E102011C6B02010E0E51
:101BC000026F0AEF16F008D03A0E0101855D04E0BD
:101BD00002011C6B0AEF16F002011C6B0201010EE0
:101BE000026F0AEF16F001018551340802E2000E7F
:101BF00001D0010E146E300E0101855D02E2000E6F
:101C000001D0010E141401E190D0300E0101855D68
:101C10000101856F01018551030DF3CFE9FFF4CF79
:101C2000EAFF8A0EE926020EEA22EE50020181192D
:101C300008E1EE500201821904E1EE50020183191D
:101C400000E100E002010F5110116FE10101855127
:101C5000030DF3CFE9FFF4CFEAFF8A0EE926020E67
:101C6000EA22EE500201815D01019F6FEE500201F8
:101C700082590101A06FEE50020183590101A16F49
:101C80000101800EA11517E09FC19FF1A0C1A0F135
:101C9000A1C1A1F10C680D680E689FC107F0A0C139
:101CA00008F0A1C109F000EC2BF004C09FF105C0C1
:101CB000A0F106C0A1F10101D890A151010A06E6E8
:101CC000000E9F5D000EA059010EA1592EE20101E8
:101CD0008551030DF3CFE9FFF4CFEAFF8A0EE92621
:101CE000020EEA22EECF14F0EECF15F0EFCF16F091
:101CF000165002018319E8AE02D0833509D00201E3
:101D00008151145C02018251155802018351165809
:101D100003E20201166903D00201010E166FF29E62
:101D20009FC10FF2A0C110F2F28E0201026B0AEF06
:101D300016F0510E0101855D37E102011C2B040EE6
:101D400002011C5D2EE1F29ED59EF29AF26AF50E1A
:101D5000F16EC00EF06E9D6AA06A9E6AA16A9F68CD
:101D6000A2685C0ED06ED568CD6ACA6A0F0EC16ECD
:101D7000946893689268929489946D926D6ADF6A10
:101D8000FF0EDF5C0BE2E868E85006E0E80600D0F2
:101D900000D000D000D0F8D7DF2AF2D700EF00F053
:101DA00002D00AEF16F006D002011C6B0201026B92
:101DB0000AEF16F0460E0101855D04E10201020EF4
:101DC000026F3AD0430E0101855D04E10201130E5A
:101DD000026F32D0520E0101855D04E10201140E42
:101DE000026F2AD0500E0101855D04E10201100E40
:101DF000026F22D0530E0101855D07E10201160E2C
:101E0000026F0201116B126B17D0540E0101855D38
:101E100007E102014B0E026F0201116B126B0CD035
:101E2000470E0101855D06E102014E0E026F0AEFC9
:101E300016F002D00201026B0AEF16F0540E0101F7
:101E4000855D04E10201490E026F48D0430E010195
:101E5000855D07E10201040E026F02010B0E016FA6
:101E60003DD0530E0101855D07E10201030E026FB3
:101E70000201080E016F32D0410E0101855D04E1BF
:101E800002014A0E026F2AD0420E0101855D07E170
:101E90000201030E026F02010A0E016F1FD0490EEC
:101EA0000101855D19E105C2AAF106C2ABF105C2C7
:101EB000AEF106C2AFF102010F51101106E0F29E21
:101EC000010E02010F6F106BF28E02019D6B9DC21D
:101ED0009EF20201026B02D00201026B0AEF16F0C1
:101EE0000101A75102E1000E01D0010E146E0101A3
:101EF000A95102E1000E01D0010E14144BE0030EB3
:101F00000101851502019F5D33E0030E0101851576
:101F100002019F6F020E02019F5D02E0000E01D0E0
:101F2000010E146E02019F5102E0000E01D0010E5D
:101F3000141008E005C2AAF106C2ABF105C2AEF169
:101F400006C2AFF102019F5106E002019D6B9DC2E6
:101F50009EF29DC29CF202019F510AE102010F51C3
:101F6000101106E0F29E010E02010F6F106BF28E4F
:101F7000030E0101851508E105C2AAF106C2ABF105
:101F800005C2AEF106C2AFF102019F0502E186EC87
:101F90001CF006D002019F5102E0000E01D0010E9C
:101FA0000201026B0AEF16F02B0E0101855D04E1C0
:101FB0000101010EA86F0BD02D0E0101855D03E11B
:101FC0000101A86904D00201026B0AEF16F00201B8
:101FD000030E026F0201090E016F0AEF16F00F0ED9
:101FE00001018515E66E020111C2E9FF12C2EAFF86
:101FF000112B000E1223270EE926020EEA22E552CB
:10200000E750EF6E0201480E111901E1125102E191
:102010000201026B230E0101855D02E10201026BE8
:102020000AEF16F0530E0101855D06E102010E0E66
:10203000026F0AEF16F009D0460E0101855D05E139
:102040000201110E026F0AEF16F002010F0E026F6D
:102050000AEF16F0F29EF28E02010F0E026F0AEFE7
:1020600016F0F29EF00E81140101A26F0F0E010115
:1020700085150101A213A2C181FFF28E02010F0E8C
:10208000026F0AEF16F00201026B0AEF16F04F0E14
:102090000101855D0EE1E66A030EE66E0101A351C2
:1020A000E66EE66A06EC18F0E552E552E552E552B6
:1020B00045D15A0E0101855D0EE1E66A030EE66E1A
:1020C0000101A551E66EE66A06EC18F0E552E5520C
:1020D000E552E55233D1460E0101855D0EE1E66A17
:1020E000030EE66E0101A451E66EE66A06EC18F0F6
:1020F000E552E552E552E55221D1530E0101855DCD
:102100000EE1E66A030EE66E02011B51E66EE66A18
:1021100006EC18F0E552E552E552E5520FD1540EA7
:102120000101855D35E101018051EA6A000FE96E28
:10213000010EEA2209C2EFFF0101802B010180514B
:10214000EA6A000FE96E010EEA220AC2EFFF0101FE
:10215000802B01018051EA6A000FE96E010EEA222C
:102160000BC2EFFF0101802B01018051EA6A000FD1
:10217000E96E010EEA220CC2EFFF0101802B010182
:102180008051EA6A000FE96E010EEA22EF6AD6D0AA
:10219000740E0101855D18E1010EE66E030EE66E18
:1021A00005C214F006C215F0166A15BE166814C0F2
:1021B000E6FF15C0E6FF16C0E6FFD6EC18F0176E76
:1021C000050EE15E1750BAD0430E0101855D0EE1A8
:1021D000E66A010EE66E02012451E66EE66A06EC3E
:1021E00018F0E552E552E552E552A8D0570E01012C
:1021F000855D0EE1E66A010EE66E02012651E66E8D
:10220000E66A06EC18F0E552E552E552E55296D042
:10221000500E0101855D11E1010EE66E060EE66EBF
:1022200081C2E6FF82C2E6FF83C2E6FFD6EC18F069
:10223000146E050EE15E145081D0410E0101855DE2
:1022400014E1010EE66E030EE66EA9C114F0156AE4
:1022500014BE156814C0E6FF15C0E6FF06EC18F0C2
:10226000E552E552E552E55269D0420E0101855D25
:1022700013E1E66A030EE66EA7C114F0156A14BEF8
:10228000156814C0E6FF15C0E6FF06EC18F0E5522D
:10229000E552E552E55252D0470E0101855D0EE14F
:1022A000E66A010EE66E02019F51E66EE66A06ECF2
:1022B00018F0E552E552E552E55240D0450E0101D5
:1022C000855D0EE1E66A030EE66E0101B251E66E2F
:1022D000E66A06EC18F0E552E552E552E5522ED0DA
:1022E000480E0101855D0EE1E66A020EE66E02010E
:1022F0000351E66EE66A06EC18F0E552E552E55247
:10230000E5521CD0490E0101855D0FE1010EE66E1C
:10231000030EE66EAEC1E6FFAFC1E6FF06EC18F0B5
:10232000E552E552E552E55209D0510E0101855DB5
:1023300005E102014C0E026F0AEF16F00201026B7A
:102340000AEF16F0350E0101855D02E3000E01D0A3
:10235000010E146E300E0101855D02E2000E01D007
:10236000010E14141CE0010EE66E060EE66E300E31
:102370000101855D030DF3CFE9FFF4CFEAFF8A0E7B
:10238000E926020EEA22EECFE6FFEECFE6FFEFCF20
:10239000E6FFD6EC18F0146E050EE15E1450020153
:1023A000026B0AEF16F04F0E0101855D07E1020195
:1023B000030E026F0201010E016F3ED0460E0101B5
:1023C000855D07E10201030E026F0201020E016F3B
:1023D00033D0530E0101855D07E10201030E026F48
:1023E0000201030E016F28D0430E0101855D04E157
:1023F0000201170E026F20D0570E0101855D04E126
:102400000201180E026F18D0500E0101855D0AE11D
:1024100002011E0E026F0201846B856B866B020146
:10242000896B0AD0510E0101855D04E102014D0E58
:10243000026F02D00201026BEDD301018551340815
:1024400002E2000E01D0010E146E300E0101855D16
:1024500002E2000E01D0010E141412E0300E010150
:10246000855D030DF3CFE9FFF4CFEAFF8A0EE9267D
:10247000020EEA2281C2EEFF82C2EEFF83C2EEFFAD
:10248000F29E300E0101855D030DF3CF85F1A68428
:10249000100E01018525A96E100E1F0B81C214F0CC
:1024A00082C215F083C216F006E0D89016321532BB
:1024B0001432E806FAE1156A166A1450A86EB0ECF8
:1024C0001AF0A684110E01018525A96E080E1F0BB6
:1024D00081C214F082C215F083C216F006E0D890D3
:1024E000163215321432E806FAE1156A166A1450EB
:1024F000A86EB0EC1AF0A684120E01018525A96E13
:1025000081C214F082C215F083C216F0156A166AF1
:102510001450A86EB0EC1AF0F28E0201026B7AD35E
:102520002B0E0101855D02E0000E01D0010E146E3C
:10253000200E0101855D02E0000E01D0010E141095
:1025400003E00201022B0CD02D0E0101855D06E196
:102550000201010E896F0201022B02D00201026BFF
:1025600059D3230E0101855D6AE1F29E84C281F296
:1025700085C282F286C283F20201895117E081C2CC
:1025800081F282C282F283C283F20C680D680E6807
:1025900081C207F082C208F083C209F000EC2BF080
:1025A00004C081F205C082F206C083F2A69EA69CFA
:1025B000A6840A0EA96E100E1F0B81C214F082C2EF
:1025C00015F083C216F006E0D89016321532143298
:1025D000E806FAE1156A166A1450A86EB0EC1AF013
:1025E000A69EA69CA6840B0EA96E080E1F0B81C288
:1025F00014F082C215F083C216F006E0D8901632AD
:1026000015321432E806FAE1156A166A1450A86EFB
:10261000B0EC1AF0A69EA69CA6840C0EA96E81C2F0
:1026200014F082C215F083C216F0156A166A1450AF
:10263000A86EB0EC1AF0F28E0201026BEBD201012F
:102640008551390802E3000E01D0010E146E300EE0
:102650000101855D02E3000E01D0010E141003E0BC
:102660000201026BD7D284C214F085C215F086C273
:1026700016F00A0E0C6E0D6A0E6A14C007F015C033
:1026800008F016C009F000EC2BF004C014F005C0EF
:1026900015F006C016F0300E0101855D176E186A40
:1026A000196A145017240201846F15501820020172
:1026B000856F165019200201866F0201022BAAD2E3
:1026C0000201026B01018551330802E3000E01D0C3
:1026D000010E146E300E0101855D02E3000E01D083
:1026E000010E141001E096D2300E0101855D020149
:1026F000266F030E02012603F35002011525E96E31
:10270000EA6AD890E936EA366F0EE926020EEA2226
:10271000EFCF21F20201226B21BF2269030E0201D9
:102720002603F35002011525E96EEA6AD890E936CE
:10273000EA366F0EE926020EEA22010EE926000EA5
:10274000EA22EFCF1FF20201206B1FBF20690201B6
:10275000136B21C21DF222C21EF2A69EA69CA68465
:10276000040EA96E26C2A8FFA5EC1AF053D20201EE
:10277000026B01018551310802E3000E01D0010E08
:10278000146E300E0101855D02E3000E01D0010ED2
:10279000141001E03FD2300E0101855D0201246F6B
:1027A0000201026BA69EA69CA684030EA96E24C2FB
:1027B000A8FFA5EC1AF02ED201018551310802E3E1
:1027C000000E01D0010E146E300E0101855D02E392
:1027D000000E01D0010E141003E00201026B1AD2A8
:1027E000300E0101855D0201176F0201120E026FAA
:1027F00011D201018551320802E3000E01D0010E11
:10280000146E300E0101855D02E3000E01D0010E51
:10281000141003E00201026BFDD1300E0101855D51
:102820000201186F0201030E026F0201016BF2D167
:10283000200E0101855D04E10201040E026F14D037
:10284000E8EC19F0000903E00201026BE3D1010199
:1028500085510201116F126B0201300E115F000EE3
:10286000125B0201040E026FD5D1200E0101855DBD
:102870000AE10201022B02010251050803E20201F2
:10288000026BC8D120D0E8EC19F0000903E0020186
:10289000026BC0D111C214F012C215F00A0E15025B
:1028A000F3CF15F00A0E1402F3CF14F0F4501526EE
:1028B000300E0101855D02011424116F000E1520F8
:1028C000126F0201022BA6D1E8EC19F0000903E017
:1028D0000201026B9FD111C214F012C215F00A0E50
:1028E0001502F3CF15F00A0E1402F3CF14F0F450D2
:1028F0001526300E0101855D02011424116F000EB2
:102900001520126F0201090E026F84D1230E0101FE
:10291000855D03E00201026B7DD10201015101E0FE
:1029200093D0F29AF29411C20FF212C210F217C2AF
:1029300016F20201165102E10201166918C215F2DF
:10294000030E02012603F35002011525E96EEA6A1F
:10295000D890E936EA366F0EE926020EEA22EFCF6A
:1029600021F20201226B21BF2269030E020126031C
:10297000F35002011525E96EEA6AD890E936EA3685
:102980006F0EE926020EEA22010EE926000EEA2267
:10299000EFCF1FF20201206B1FBF2069A3C113F20A
:1029A00002010F51101141E10201136BA6840A0EBE
:1029B000A96E100E1F0B81C214F082C215F083C2E3
:1029C00016F006E0D890163215321432E806FAE115
:1029D000156A166A1450A86EA5EC1AF0A6840B0EA0
:1029E000A96E080E1F0B81C214F082C215F083C2BB
:1029F00016F006E0D890163215321432E806FAE1E5
:102A0000156A166A1450A86EA5EC1AF0A6840C0E6E
:102A1000A96E81C214F082C215F083C216F0156A45
:102A2000166A1450A86EA5EC1AF0020115510201A5
:102A3000235D08E021C21DF222C21EF215C223F25C
:102A400016C225F2F28AE0D00201010521E102015D
:102A5000FF0E115D000E125902E3000E01D0010EAF
:102A6000146E0201000ED8801155000E125502E3BB
:102A7000000E01D0010E14140AE011C2A3F1A69EAB
:102A8000A69CA684A96AA3C1A8FFA5EC1AF0BCD095
:102A9000020E0201015D22E10201FF0E115D000E36
:102AA000125902E3000E01D0010E146E0201000E55
:102AB000D8801155000E125502E3000E01D0010E10
:102AC00014140BE011C2A4F1A69EA69CA684010ECC
:102AD000A96EA4C1A8FFA5EC1AF096D0030E0201BE
:102AE000015D22E10201FF0E115D000E125902E3A9
:102AF000000E01D0010E146E0201000ED880115597
:102B0000000E125502E3000E01D0010E14140BE06A
:102B100011C21BF2A69EA69CA684020EA96E1BC221
:102B2000A8FFA5EC1AF070D0080E0201015D17E1B4
:102B30000201FF0E115D000E125910E211C2A7F141
:102B40000101A75102E102019F6BA69EA69CA684EB
:102B50000E0EA96EA7C1A8FFA5EC1AF055D0090E5C
:102B60000201015D26E10201650E115D000E1259A0
:102B70001FE2A8C114F0156A14BE156811C208F04E
:102B800012C209F014C00DF015C00EF0E2EC2AF0EC
:102B900006C0A9F10101A95102E102019F6BA69EA5
:102BA000A69CA6840F0EA96EA9C1A8FFA5EC1AF0D9
:102BB0002BD00A0E0201015D12E10201FF0E115D30
:102BC000000E12590BE211C2B2F1A69EA69CA68479
:102BD000050EA96EB2C1A8FFA5EC1AF015D00B0E18
:102BE0000201015D11E102014C0E115D000E12594E
:102BF0000BE211C203F2A69EA69CA6841F0EA96E2C
:102C000003C2A8FFA5EC1AF00201026B03D0020177
:102C1000026B00D00101822B010181510101825D13
:102C200002E10201006B0201A35111E10101805197
:102C300000080DE280C1E6FF000EE66E010EE66EB2
:102C400003EC29F0E552E552E5520101806BA1EC5D
:102C500029F0E552E552E7CFD9FF1200D9CFE6FFC0
:102C6000E1CFD9FF020EE126FD0EDBCFDEFFDBCF89
:102C7000DDFFDECFF6FFDDCFF7FF0800F5500FE0F8
:102C8000DFCFF6FFDF2A010EDBCFF7FF01E3DB2A00
:102C90000800F550E66E44EC0CF0E552EAD7020E5F
:102CA000E15C02E2E16AE552E16EE552E7CFD9FF6D
:102CB0001200D9CFE6FFE1CFD9FF050EE126FD0EC8
:102CC000DBCFDEFFDBCFDDFFFB0EDB5023E0FD0EB5
:102CD000DBCF14F0FE0EDBCF15F00001800E1514D3
:102CE00014E02D0EE66E44EC0CF0E552086809681D
:102CF000FD0EDBCF0DF0FE0EDBCF0EF0B5EC2AF0B3
:102D000006C0DEFF07C0DDFF05D02B0EE66E44ECEB
:102D10000CF0E552FC0EDB50E76E040EE7CFDBFF54
:102D2000FC0EDB50010A15E0030A11E0010A0DE078
:102D3000070A17E0010A15E1100EF36E020EF3CF39
:102D4000DBFF270EF36E030E13D0640E03D00A0EC2
:102D500001D0010EF36E020EF3CFDBFF030EDB6A30
:102D600009D0E80EF36E020EF3CFDBFF030EF36E15
:102D7000F3CFDBFF040EDB5000083BE2000EDFCF99
:102D800008F0010EDBCF09F0020EDBCF0DF0030ED1
:102D9000DBCF0EF081EC2CF00850300FE66E44ECE7
:102DA0000CF0E552000EDFCF08F0010EDBCF09F08A
:102DB000020EDBCF0DF0030EDBCF0EF081EC2CF01A
:102DC00004C0DEFF05C0DDFFD950020FE96EDACF87
:102DD000EAFF0A0E0D6E0E6AEECF08F0EDCF09F095
:102DE00081EC2CF008C0EEFF09C0EDFF040EDB06FD
:102DF000C1D7050EE15C02E2E16AE552E16EE552FF
:102E0000E7CFD9FF1200D9CFE6FFE1CFD9FF070EF8
:102E1000E126D9CFE9FFDACFEAFFFC0EDBCFEEFFE8
:102E2000FD0EDBCFEEFFFE0EDBCFEEFFFA0EDB502A
:102E300039E0D950FC0FE96EFF0EDA20EA6E020E7F
:102E4000D890EB50000A06E6000EEE5C000EEE583D
:102E5000000EEF5822E22D0EE66E44EC0CF0E55227
:102E6000FC0EDBCF14F0FD0EDBCF15F0FE0EDBCF3A
:102E700016F00C680D680E6814C007F015C008F055
:102E800016C009F000EC2BF004C0DFFF010E05C0F6
:102E9000DBFF020E06C0DBFF05D02B0EE66E44EC16
:102EA0000CF0E552FB0EDB50E76E060EE7CFDBFFC2
:102EB000FB0EDB50010A25E0030A21E0010A1DE0B8
:102EC000070A27E0010A12E0030A23E1A00EF36ECD
:102ED000030EF3CFDBFF860EF36E040EF3CFDBFFA2
:102EE000010EF36E050EF3CFDBFF1ED0100EF36E56
:102EF000030EF3CFDBFF270E11D0640E03D00A0EB2
:102F000001D0010EF36E030EF3CFDBFF040EDB6A7C
:102F100009D0E80EF36E030EF3CFDBFFF36E040E61
:102F2000F3CFDBFF050EDB6A060EDB50000864E220
:102F3000DFCF14F0010EDBCF15F0020EDBCF16F061
:102F400014C007F015C008F016C009F0030EDBCF5F
:102F50000CF0040EDBCF0DF0050EDBCF0EF088EC8D
:102F60002AF00750300FE66E44EC0CF0E552DFCF4C
:102F700014F0010EDBCF15F0020EDBCF16F014C0FB
:102F800007F015C008F016C009F0030EDBCF0CF0F7
:102F9000040EDBCF0DF0050EDBCF0EF00EC0F5FFFB
:102FA00088EC2AF0F5AE06D0000E036C041E042255
:102FB000051E052203C0DFFF010E04C0DBFF020E69
:102FC00005C0DBFFD950030FE96EDACFEAFF0A0E26
:102FD0000C6E0D6A0E6AEECF07F0EECF08F0EFCF61
:102FE00009F088EC2AF009C0EDFF08C0EDFF07C02A
:102FF000EFFF060EDB0698D7070EE15C02E2E16AFE
:10300000E552E16EE552E7CFD9FF1200D9CFE6FFD6
:10301000E1CFD9FF050EE126FD0EDBCFDEFFDBCFD2
:10302000DDFFFB0EDB503AE0FD0EDBCF14F0FE0EB1
:10303000DBCF15F0800E151420E001018051EA6A03
:10304000000FE96E010EEA222D0EEF6E802B8051EB
:10305000EA6A000FE96E010EEA22EF6A0868096861
:10306000FD0EDBCF0DF0FE0EDBCF0EF0B5EC2AF03F
:1030700006C0DEFF07C0DDFF11D001018051EA6A02
:10308000000FE96E010EEA222B0EEF6E802B8051AD
:10309000EA6A000FE96E010EEA22EF6AFC0EDB50CD
:1030A000E76E040EE7CFDBFFFC0EDB50010A15E0F4
:1030B000030A11E0010A0DE0070A17E0010A15E111
:1030C000100EF36E020EF3CFDBFF270EF36E030E2E
:1030D00013D0640E03D00A0E01D0010EF36E020E5F
:1030E000F3CFDBFF030EDB6A09D0E80EF36E020EAE
:1030F000F3CFDBFF030EF36EF3CFDBFF040EDB50E9
:1031000000084AE2000EDFCF08F0010EDBCF09F025
:10311000020EDBCF0DF0030EDBCF0EF081EC2CF0B6
:103120000850300FE66E01018051EA6A000FE96E27
:10313000010EEA22E552E750EF6E802B8051EA6AD9
:10314000000FE96E010EEA22EF6A000EDFCF08F0F1
:10315000010EDBCF09F0020EDBCF0DF0030EDBCF4B
:103160000EF081EC2CF004C0DEFF05C0DDFFD9506D
:10317000020FE96EDACFEAFF0A0E0D6E0E6AEECF8D
:1031800008F0EDCF09F081EC2CF008C0EEFF09C08B
:10319000EDFF040EDB06B2D7050EE15C02E2E16A48
:1031A000E552E16EE552E7CFD9FF1200D9CFE6FF35
:1031B000E1CFD9FF070EE126D9CFE9FFDACFEAFF49
:1031C000FC0EDBCFEEFFFD0EDBCFEEFFFE0EDBCF06
:1031D000EEFFFA0EDB5043E0D950FC0FE96EFF0E14
:1031E000DA20EA6E020ED890EB50000A06E6000ED6
:1031F000EE5C000EEE58000EEF5827E20101805100
:10320000EA6A000FE96E010EEA222D0EEF6E802BA6
:10321000FC0EDBCF14F0FD0EDBCF15F0FE0EDBCF86
:1032200016F00C680D680E6814C007F015C008F0A1
:1032300016C009F000EC2BF004C0DFFF010E05C042
:10324000DBFF020E06C0DBFF0AD001018051EA6AF3
:10325000000FE96E010EEA222B0EEF6E802BFB0EA3
:10326000DB50E76E060EE7CFDBFFFB0EDB50010AFB
:1032700025E0030A21E0010A1DE0070A27E0010A10
:1032800012E0030A23E1A00EF36E030EF3CFDBFF7F
:10329000860EF36E040EF3CFDBFF010EF36E050E08
:1032A000F3CFDBFF1ED0100EF36E030EF3CFDBFF68
:1032B000270E11D0640E03D00A0E01D0010EF36E5A
:1032C000030EF3CFDBFF040EDB6A09D0E80EF36ECA
:1032D000030EF3CFDBFFF36E040EF3CFDBFF050E1F
:1032E000DB6A060EDB50000869E2DFCF14F0010E46
:1032F000DBCF15F0020EDBCF16F014C007F015C0BF
:1033000008F016C009F0030EDBCF0CF0040EDBCF83
:103310000DF0050EDBCF0EF02DEC2CF00750300F2A
:10332000E66E01018051EA6A000FE96E010EEA22A1
:10333000E552E750EF6E802B8051EA6A000FE96E8C
:10334000010EEA22EF6ADFCF14F0010EDBCF15F099
:10335000020EDBCF16F014C007F015C008F016C03F
:1033600009F0030EDBCF0CF0040EDBCF0DF0050EE1
:10337000DBCF0EF02DEC2CF003C0DFFF010E04C0FC
:10338000DBFF020E05C0DBFFD950030FE96EDACF79
:10339000EAFF0A0E0C6E0D6A0E6AEECF07F0EECF52
:1033A00008F0EFCF09F02DEC2CF009C0EDFF08C0BC
:1033B000EDFF07C0EFFF060EDB0693D7070EE15CBB
:1033C00002E2E16AE552E16EE552E7CFD9FF120071
:1033D00001018551390802E3000E01D0010E146E7F
:1033E000300E855D02E3000E01D0010E14101200B4
:1033F0000201A051A11110E10E51146E156AC80E00
:10340000141806E1155004E1F40EA06F010E03D06C
:10341000100EA06F270EA16FA007000EA15B6DA27A
:1034200007D0A051A1112EE1897089B013D027D007
:103430000101B55102E1899022D0B50502E18980F0
:1034400009D0020EB55D02E1898019D0040EB55D88
:1034500003E1899089821200100EB55D06E1020138
:10346000A051A1110FE189700AD0200EB55D0AE1CB
:103470000201A051A11106E1897089A002D08992B0
:1034800012008982120012001200120012001FEFB7
:1034900028F012006FEF28F06D840101080EB36F61
:1034A000070EB46FB307000EB45BB351B411FAE169
:1034B0006D941200D9CFE6FFE1CFD9FFFD0EDBCF2F
:1034C00008F0FE0EDBCF09F0720E081801E109507A
:1034D00033E0E868081802E17F0E09182BE0740E4B
:1034E000081801E1095024E0750E081801E109509F
:1034F0001DE0730E081801E1095016E0030E0818CC
:1035000001E109500FE0020E081801E1095008E03E
:10351000010E081801E1095001E010D0BBDF0FD007
:10352000B8DF0DD0B4DF0BD0B0DF09D0ACDF07D0EF
:10353000ABDF05D0ABDF03D0000001D000D0010E1F
:1035400000D0E552E7CFD9FF1200F29E550EA76ECC
:10355000AA0EA76EA682F28EA6B2FED7A69412007D
:10356000550EA76EAA0EA76EA682A6B2FED7A69487
:103570001200D9CFE6FFE1CFD9FF040EE1268A98E9
:103580000101926B080E925D2DE2F29E8A98FE0E6A
:10359000DBA00DD09398180EDF6EDF06FEE1938856
:1035A000DE52960EDD6E010EDB0611E0FCD793981D
:1035B000B40EF36E020EF3CFDBFFDB06FEE1938861
:1035C000180EF36E030EF3CFDBFFDB06FEE1F28E87
:1035D000FE0EDBCFF3FFF390F342F3CFDBFF0101ED
:1035E000922BD0D7040EE15C02E2E16AE552E16E73
:1035F000E552E7CFD9FF1200D9CFE6FFE1CFD9FFDF
:10360000020EE1268A980101956B966B0101926B7F
:10361000080E0101925D35E2F29E8A9893980000AF
:10362000000000000000000000000000000000009A
:10363000000000000000000000000000000000008A
:1036400000009388140EDF6EDF0602E0FDD7FCD782
:10365000D89001019633953381A803D00101958F4D
:1036600004D00101959F0101966BF28EDE52640E2B
:10367000DD6E010EDB0602E0FCD7FBD70101922BC9
:10368000C7D795C1F3FF96C1F4FF00D0020EE15CED
:1036900002E2E16AE552E16EE552E7CFD9FF12009E
:1036A000D9CFE6FFE1CFD9FF150EE12693880000C0
:1036B000000000000000000000000000000000000A
:1036C00000000000000000000000000000000000FA
:1036D000000000000000000000000000000081B8B1
:1036E00003D0F36AF46AE5D093988A989398780E99
:1036F000DF6EDF0602E0FDD7FCD7DE52780EDD6E0E
:10370000010EDB0602E0FCD7FBD7780EF36E020E4B
:10371000F3CFDBFF020EDB0602E0FCD7FBD7780E0F
:10372000F36E030EF3CFDBFF030EDB0602E0FCD7E4
:10373000FBD7780EF36E040EF3CFDBFF040EDB062F
:1037400002E0FCD7FBD7780EF36E050EF3CFDBFF5C
:10375000050EDB0602E0FCD7FBD7780EF36E060EF3
:10376000F3CFDBFF060EDB0602E0FCD7FBD7780EBB
:10377000F36E070EF3CFDBFF070EDB0602E0FCD78C
:10378000FBD7780EF36E080EF3CFDBFF080EDB06D7
:1037900002E0FCD7FBD7780EF36E090EF3CFDBFF08
:1037A000090EDB0602E0FCD7FBD7F29E9388960E4B
:1037B000F36E0A0EF3CFDBFF0A0EDB0602E0FCD746
:1037C000FBD78150100B01E0010E0101956F966B44
:1037D000F28E780EF36E0B0EF3CFDBFF0B0EDB06D3
:1037E00002E0FCD7FBD7780EF36E0C0EF3CFDBFFB5
:1037F0000C0EDB0602E0FCD7FBD7780EF36E0D0E45
:10380000F3CFDBFF0D0EDB0602E0FCD7FBD7780E13
:10381000F36E0E0EF3CFDBFF0E0EDB0602E0FCD7DD
:10382000FBD7780EF36E0F0EF3CFDBFF0F0EDB0628
:1038300002E0FCD7FBD7780EF36E100EF3CFDBFF60
:10384000100EDB0602E0FCD7FBD7780EF36E110EEC
:10385000F3CFDBFF110EDB0602E0FCD7FBD7780EBF
:10386000F36E120EF3CFDBFF120EDB0602E0FCD785
:10387000FBD7780EF36E130EF3CFDBFF130EDB06D0
:1038800002E0FCD7FBD7780EF36E140EF3CFDBFF0C
:10389000140EDB0602E0FCD7FBD70101955196110F
:1038A00004E0F36AF46A05D004D0010EF36EF46A02
:1038B00000D0150EE15C02E2E16AE552E16EE552EC
:1038C000E7CFD9FF1200D9CFE6FFE1CFD9FFFE0E37
:1038D000DBCF15F0800E151407E1FD0EDBCF14F0E1
:1038E000FE0EDBCF15F00AD0FD0EDBCF14F0FE0E7E
:1038F000DBCF15F0146C151E000E152214C0F3FF5B
:1039000015C0F4FFE552E7CFD9FF1200880E02017F
:1039100005190FE1FC0E06190CE105C2AEF106C255
:10392000AFF105C2AAF106C2ABF19E6B9EC29DF239
:103930000FD0880E0101AE190BE1FC0EAF1908E1A2
:1039400005C2AEF106C2AFF105C2AAF106C2ABF1E3
:10395000880E0201051905E1FC0E061902E1000EB0
:1039600001D0010E146E880E0101AA1905E1FC0EAA
:10397000AB1902E1000E01D0010E141401E1CAD00E
:1039800002019D5101E0ADD00101A75102E1000EFD
:1039900001D0010E146EA95102E1000E01D0010EFA
:1039A000141401E1B7D0020105510101AE1904E17F
:1039B000020106510101AF1904E0AEC1AAF1AFC185
:1039C000ABF1AA510201055D166E06510101AB551E
:1039D000176E16C0E6FFE66E76DFE552E552F3CFCE
:1039E00014F0F4CF15F0F3CFE6FFF4CFE6FFA9C152
:1039F0001AF01B6A1ABE1B681AC0E6FF1BC0E6FF5E
:103A000062DFE552E552E552E7CF15F0E552E7CF28
:103A100014F0F3CF18F0F4CF19F01550F418E8AE05
:103A200002D0193404D01850145C1950155872E3A0
:103A300005C2AEF106C2AFF1F29EA7C118F0196A35
:103A400018BE1968A9C116F0176A16BE17680101D9
:103A5000AA510201055D146E06510101AB55156EA8
:103A600014C008F0096E16C00DF017C00EF062EC1D
:103A70002AF018C00DF019C00EF0B5EC2AF006C0FF
:103A80009DF107C09EF10101800E071406E09D6DB7
:103A90009E1F000E9E23B16902D0010EB16FF28EFF
:103AA000B25110E0B1510201165D0DE0F29E01012C
:103AB000B25102010F6F106BA3C113F2F28E010E0F
:103AC0009E6F0CD002019E6BF29E9DC10FF29EC1B3
:103AD00010F2B1C116F2A3C113F2F28E010E9D6F66
:103AE00012009E5113E00F51101114E19E6BF29ED3
:103AF0000101B2519D2502010F6F000E01019E21AF
:103B00000201106FB1C116F2F28E12000F511011A6
:103B100001E19D6B120002010E510D0A6BE0040AD7
:103B200063E0030A61E0010A5FE0070A5DE0040A5E
:103B300057E00F0A51E0010A4AE0030A46E0010A91
:103B40003EE0070A30E0010A1FE0030A3EE0010AF6
:103B500003E0C80A01E0BFD1A3DDF350F41004E094
:103B60000201010E0E6FB8D10201C80E0E6F0101E5
:103B7000380E8E6F8D6F8C6F2D0E8B6F0201880E3D
:103B8000056FFC0E066FA3D1440EE66EF2DCE55223
:103B900002010E2B0101976B986B996B9A6BF29E49
:103BA0009B6B9C6B0AD0F29E0101DC0ED8809B556A
:103BB000050E9C5502E202010E2BF28E8DD170DDB6
:103BC000F3CF95F1F4CF96F112D0CC0E01D0BE0E0A
:103BD000E66ECFDCE5520BD00FDDF3CF8FF107D0CF
:103BE0000BDDF3CF90F103D007DDF3CF93F10201AA
:103BF0000E2B72D101DDF3CF94F101012B0E8B6FEF
:103C0000905105E08F1D8F6F8F2B2D0E8B6F8F5175
:103C1000956F966B300E8E6F8FC114F00001156A90
:103C2000010E14161450151003E00101350E8E6FAD
:103C3000010E0F0B010105E0D89096339533E8068D
:103C4000FBE195C114F096C115F00A0E0D6E0E6AD7
:103C500095C108F096C109F081EC2CF004C014F075
:103C600005C015F0300E042401018D6F0A0E0D6E93
:103C70000E6A95C108F096C109F081EC2CF008C0DD
:103C800095F109C096F108C014F009C015F00A0EAC
:103C90000D6E0E6A81EC2CF0300E042401018C6F45
:103CA00002010E6B166E176A16BE1768300E165E8E
:103CB000000E175A640E1702F3CF17F01602F3CF57
:103CC00016F0F45017268DC118F0196A18BE19683D
:103CD000300E185E000E195A0A0E1902F3CF19F0B1
:103CE0001802F3CF18F0F45019261650F324146E6E
:103CF00017501920156E8EC11AF01B6A1ABE1B6868
:103D0000300E1A5E000E1B5A14501A240101AC6FBB
:103D100015501B20AD6F2D0E8B5D04E1AC6DAD1FFA
:103D2000000EAD23AC51020107270101AD51020184
:103D30000823042B0351045D01E0CED00451146E1E
:103D4000156A04C20DF015C00EF007C208F008C2D3
:103D500009F062EC2AF008C007F209C008F208C0B6
:103D600005F209C006F208C0E6FF09C0E6FFABDDB8
:103D7000E552E552F3CF07F2F4CF08F2A9C11AF0E9
:103D80001B6A1ABE1B681AC0E6FF1BC0E6FF9BDD5C
:103D9000E552E552F3CF18F0F4CF19F0F3CFE6FF78
:103DA000F4CFE6FF07C2E6FF08C2E6FF8CDDE5526E
:103DB000E552E552E7CF19F0E552E7CF18F0F3CF1F
:103DC00016F0F4CF17F0F3CF08F0F4CF09F018C0D5
:103DD0000DF019C00EF062EC2AF019AE04D0046C9C
:103DE000051E000E052204C014F005C015F004C025
:103DF000E6FF05C0E6FFA9C11EF01F6A1EBE1F68D0
:103E00001EC0E6FF1FC0E6FF5EDDE552E552E5524B
:103E1000E7CF15F0E552E7CF14F0F3CF1CF0F4CF65
:103E20001DF0020E0D6E0E6AF3CF08F0F4CF09F00C
:103E300062EC2AF008C01CF009C01DF009501518EA
:103E4000E8AE02D0153404D014501C5C15501D5837
:103E5000020E166E0E6EA9C109F048EC2AF009C0D8
:103E600014F0156A14BE156814C0E6FF15C0E6FF0D
:103E70002ADDE552E552F35002010727F4500823EA
:103E8000050E0D6E0E6A07C208F008C209F062EC5A
:103E90002AF008C007F209C008F20201050E080363
:103EA000F3CF08F20703F3CF07F2F4500827800E90
:103EB000061509E007C205F208C206F2056D061FE5
:103EC000000E062304D007C205F208C206F2076BF3
:103ED000086B046B01D00E6B8BC109F28CC10AF226
:103EE0008DC10BF28EC10CF28CC116F0176A16BE92
:103EF0001768300E165E000E175A640E1702F3CFC5
:103F000017F01602F3CF16F0F45017268DC118F0F3
:103F1000196A18BE1968300E185E000E195A0A0E7A
:103F20001902F3CF19F01802F45019261650F32491
:103F3000146E17501920156E8EC11AF01B6A1ABE26
:103F40001B68300E1A5E000E1B5A14501A24010111
:103F5000AC6F15501B20AD6F2D0E8B5D04E1AC6D69
:083F6000AD1F000EAD2312009D
:083F6800D9CFE6FFE1CFD9FF3C
:103F7000E652A09A6A6A686A160E6F6E9F0E6B6EA2
:103F80007B0E696E6D8C6E6A030EE66EE66AE66AFB
:103F9000710EE66E0F0EE66E67EC2CF0146E050ED9
:103FA000E15E14506D9CDF6ADF50146E156A100ECE
:103FB000145C000E155810E2DF50040DF3CFE9FF3A
:103FC000F4CFEAFF000EE926040EEA22EE6AEE6A5A
:103FD000EE6AEE6ADF2AE8D7160E706E68A602D087
:103FE0006896FCD70101D06BD56BD66BD76B6D98FB
:103FF000DF6A040EDF5C18E2EA6ADF34FE0BEA36A1
:10400000E96EC40EE926010EEA22EE6AED6AEA6A5A
:10401000DF34FE0BEA36E96EBC0EE926010EEA2219
:10402000EE6AED6ADF2AE5D70101080EC46F040EBF
:10403000C56FB66BB56BE552E552E7CFD9FF1200FD
:10404000D9CFE6FFE1CFD9FFE6520101B50507E17F
:104050006DBA05D0686A69806988020EB56F6850CC
:10406000040B05E06950040B02E06894B7D86DB208
:104070005FD06850010B16E06950010B13E074DF4C
:10408000D08EA28AA08AF28E0101040EB56F0401BF
:10409000400E026F040E036F080E016F006B8C0E52
:1040A000001368906850100B05E06950100B02E097
:1040B00083D868986850400B13E06950400B10E0BB
:1040C000010EE66EE66A000EE66EE66A730EE66EB6
:1040D000E66A5AEC1AF0146E060EE15E1450689C03
:1040E0006850200B04E06950200B01E04CD8685068
:1040F000020B13E06950020B10E0010EE66EE66A57
:10410000000EE66EE66AE6687F0EE66E5AEC1AF07E
:10411000146E060EE15E14506A6A040E0101E76E29
:10412000B519E8AE02D0E73402D0E750B55D02E23F
:10413000A19A24D069A621D0DF6A040EDF5C1DE2BB
:1041400068A61BD06CCFDDF16896780E0101DD15F5
:1041500002E159D810D0000EE66EE66ADD0EE66E7A
:10416000010EE66E720EE66EE66A5AEC1AF0146EF6
:10417000060EE15E1450DF2AE0D7A19AE552E5521F
:10418000E7CFD9FF120070A015D0B8C1E9FFB9C1BF
:10419000EAFFEF5080080DE1C4C1E9FFC5C1EAFFA5
:1041A000EF50840806E1B8C1E9FFB9C1EAFF8C0EFF
:1041B000EF6E7090689A1200698468986D82000EA4
:1041C000E66EE66AE66EE66A750EE66EE66A5AEC3A
:1041D0001AF0146E060EE15E14501200000EE66E28
:1041E000E66AE66EE66A740EE66EE66A5AEC1AF065
:1041F000146E060EE15E14506D92699468A402D0AC
:104200006894FCD71200D9CFE6FFE1CFD9FFE65280
:10421000FD0E0101DD155AE17E0EDD15E8407F0B34
:10422000040DF3CFB8F1F4CFB9F1000EB827040EA6
:10423000B923B8C1BAF1B9C1BBF1BA75B8C1E9FFC8
:10424000B9C1EAFFEF503C0BE842E8420D083CE1FF
:10425000B8C1E9FFB9C1EAFF020EE926000EEA2261
:10426000EECF14F0EFCF15F0480E14182BE1040E2A
:10427000151828E1B8C1E9FFB9C1EAFF020EE92625
:10428000000EEA22400EEE6E040EED6EDF6ADF5085
:10429000146E156A080E145C000E155813E2DF50F8
:1042A000EA6A480FE96E040EEA22EF50E66EDF502C
:1042B000EA6A400FE96E040EEA22E552E750EF6E1B
:1042C000DF2AE5D70DD807D02ED805D0FD0EDD1595
:1042D000040801E14ED8E552E552E7CFD9FF1200BC
:1042E000C4C1E9FFC5C1EAFFEF50800B05E0C4C1BE
:1042F000E9FFC5C1EAFFEF6A0101CC6BCD6BD16B61
:10430000D26BD06BB2D8000EE66EE66AE66EE66A55
:10431000030EE66EE66A5AEC1AF0146E060EE15EC3
:104320001450CAEF23F0020E0101CD5D02E125EF2A
:1043300025F069D80101DE511AE1BAC1E9FFBBC11C
:10434000EAFFEE52080EEF6EBAC1E9FFBBC1EAFF09
:10435000020EE926000EEA22400EEE6E040EED6E0D
:10436000BAC1E9FFBBC1EAFF8C0EEF6E1200DE6B33
:104370001200D9CFE6FFE1CFD9FFE652C4C1E9FF71
:10438000C5C1EAFFEF50400B01E0010EDF6E0101F5
:10439000C475080EB55D09E142C46EFF6E50000899
:1043A00002E2100E01D0040EB56FCD0526E1C4C1A6
:1043B000E9FFC5C1EAFF020EE926000EEA22480E17
:1043C000EE6E040EED6EB8DA020E0101CC5D06E170
:1043D000C4C1E9FFC5C1EAFF840E0DD0DF5006E17C
:1043E000C4C1E9FFC5C1EAFFC80E05D0C4C1E9FFD9
:1043F000C5C1EAFF880EEF6E01D005D8E552E5523F
:10440000E7CFD9FF1200D9CFE6FFE1CFD9FF020EE7
:10441000E1260101CD6BC4C1E9FFC5C1EAFFEF6A26
:10442000040EC419146EC5C115F0DE6EC5C1DDFFE2
:10443000DECFE9FFDDCFEAFFEF6AD5AF0CD0D85170
:10444000D91107E005D0D9C1FAFF0101D851F96EA1
:10445000FADF0101D59F020EE15C02E2E16AE5525A
:10446000E16EE552E7CFD9FF120004014051600B25
:10447000E842E842E842E842E842000901E012006E
:1044800041510C0A50E00B0A3FE00C0A31E0010AEE
:1044900022E00B0A1EE0020A1CE0030A18E0080AE8
:1044A00010E0010A0CE00F0A08E0030A01E0120024
:1044B0000101D08F080EB56F120019EF23F0C1EF84
:1044C00025F00101B60ECE6F010ECF6F0CD070EF4C
:1044D00023F094EF22F044510101CE6FCF6BB70E61
:1044E000CE27010ECF23D081010ED16FD08F1200C5
:1044F0000101D08F04014451EA6AB70FE96E010E41
:10450000EA2242C4EFFF1200000EE66EE66AE66E93
:10451000E66A020EE66EE66A5AEC1AF0146E060EB1
:10452000E15E145012001200D9CFE6FFE1CFD9FFAF
:10453000040EE1260401420510E140511F0B000961
:104540000CE10101D08F030E0401415D04E1010182
:10455000010EDC6F02D00101DC6B040142515FE10E
:1045600040511F0B02085BE144510F0B000957E05B
:104570000101D08F040144BF0BD044510F0BE96EF1
:10458000EA6AD890E936EA36BC0EE926010E0AD06E
:1045900044510F0BE96EEA6AD890E936EA36C40E48
:1045A000E926010EEA22EECFDEFFEDCFDDFF030E9E
:1045B000415D06E1DECFE9FFDDCFEAFF840E2ED0BC
:1045C00044510F0B156A700F146E0F0E1522020E58
:1045D00014C0DBFF030E15C0DBFF020EDBCFE9FFCB
:1045E000030EDBCFEAFFEF9044AF0CD0DECFE9FF44
:1045F000DDCFEAFFEF6ADF74DECFE9FFDDCFEAFF50
:10460000400E0CD0DECFE9FFDDCFEAFF880EEF6E63
:10461000DF74DECFE9FFDDCFEAFFC80EEF6E040ED8
:10462000E15C02E2E16AE552E16EE552E7CFD9FFD3
:104630001200800E0401405D52E10101C00ED06FF6
:1046400004014351030A29E0010A09E0030A45E194
:104650000101920ECE6F560ECF6F120E38D042511E
:10466000F66EF76AD890F636F736690EF626570ECC
:10467000F7220900F5CFCEF10A00F5CFCFF1020EF7
:104680000101F76ACE25F66ECF51F7220900F5CF6A
:10469000D1F10A00F5CFD2F11200040E425D1AE208
:1046A0004251F66EF76AD890F636F7366B0EF6265C
:1046B000570EF7220900F5CFCEF10A00F5CFCFF162
:1046C000CEC1F6FFCFC1F7FF0800F5500101D16F51
:1046D000D26B12000101D06B12000101D06B1200ED
:1046E000D9CFE6FFE1CFD9FF020EE1260401486BE6
:1046F000496B40511F0B020A11E0030A0CE0010A4A
:1047000035E10101D08F040148810101DC052EE172
:10471000040148832BD00101D08F28D00101D08F14
:10472000040144BF0BD044510F0BE96EEA6AD890E4
:10473000E936EA36BC0EE926010E0AD044510F0BC9
:10474000E96EEA6AD890E936EA36C40EE926010E27
:10475000EA22EECFDEFFEDCFDDFFDECFE9FFDDCFDA
:10476000EAFFEF50040B02E0010E486F0101D0AFE9
:1047700007D0480ECE6F040ECF6FD081020ED16FDE
:10478000020EE15C02E2E16AE552E16EE552E7CF3A
:10479000D9FF12006D980101D0BF47D0D5AF26D008
:1047A000020ECD6FC4C1E9FFC5C1EAFFEE52EF6A48
:1047B000C4C1E9FFC5C1EAFFC80EEF6EBAC1E9FF87
:1047C000BBC1EAFFEE52080EEF6EBAC1E9FFBBC1F2
:1047D000EAFF020EE926000EEA22480EEE6E040EF3
:1047E000ED6EBAC1E9FFBBC1EAFF7AD0BAC1E9FFF9
:1047F000BBC1EAFFEE52080EEF6EBAC1E9FFBBC1C2
:10480000EAFF020EE926000EEA22400EEE6E040ECA
:10481000ED6EBAC1E9FFBBC1EAFF8C0EEF6EC4C1F9
:10482000E9FFC5C1EAFF840E5CD0D5BF84D0040186
:1048300040AF59D00101D1510401465D0101D2516F
:104840000401475904E246C4D1F147C4D2F174D8F7
:104850000101010ECD6FBAC1E9FFBBC1EAFFEE5203
:10486000080EEF6EBAC1E9FFBBC1EAFF020EE926EE
:10487000000EEA22400EEE6E040EED6EBAC1E9FFA4
:10488000BBC1EAFF800EEF6EDE6BB8C1E9FFB9C1B4
:10489000EAFFEE52080EEF6EB8C1E9FFB9C1EAFFB8
:1048A000020EE926000EEA22400EEE6E040EED6EB8
:1048B000B8C1E9FFB9C1EAFF840EEF6E010EDE6FE9
:1048C000C4C1E9FFC5C1EAFF020EE926000EEA22D3
:1048D000480EEE6E040EED6EC4C1E9FFC5C1EAFFDD
:1048E000C80EEF6E12000101020ECD6FC4C1E9FFC8
:1048F000C5C1EAFFEE52EF6AC4C1E9FFC5C1EAFFD4
:10490000C80EEF6EBAC1E9FFBBC1EAFFEE52080E56
:10491000EF6EBAC1E9FFBBC1EAFF020EE926000E45
:10492000EA22480EEE6E040EED6EBAC1E9FFBBC17D
:10493000EAFFC80EEF6E1200D9CFE6FFE1CFD9FF34
:10494000020EE1260101080ED15D000ED2590DE2E2
:10495000D1C1DEFFD2C1DDFFCC5102E1010E03D097
:10496000CC0506E1020ECC6F03D0080EDE6EDD6AC8
:10497000C4C1E9FFC5C1EAFFEF92C4C1E9FFC5C1E7
:10498000EAFFEF90C4C1E9FFC5C1EAFF010EDB50A9
:10499000EF12C4C1E9FFC5C1EAFFEE52DFCFEFFF5E
:1049A000000EDB50D15F010EDB50D25B480EDA6F98
:1049B000040EDB6FD0B120D0D9CFE9FFDACFEAFF08
:1049C000EE50ED1038E0CEC1F6FFCFC1F7FFCE2B91
:1049D000000ECF230800F550E66EDAC1E9FFDBC117
:1049E000EAFFDA2B000EDB23E552E750EF6EDF061D
:1049F000010EE2E2DB06E0D7D9CFE9FFDACFEAFF2A
:104A0000EE50ED1018E0CEC1E9FFCFC1EAFFCE2B8A
:104A1000000ECF23EF50E66EDAC1E9FFDBC1EAFFFB
:104A2000DA2B000EDB23E552E750EF6EDF06010EB6
:104A3000E3E2DB06E1D7020EE15C02E2E16AE55265
:104A4000E16EE552E7CFD9FF1200D9CFE6FFE1CF03
:104A5000D9FF020EE126B8C1E9FFB9C1EAFFEE5263
:104A6000EFCFDFFFDFCF14F014500101D65D000E51
:104A7000D75902E2D6C1DFFFDF50146E156AE85045
:104A8000D65DD66F1550D759D76F010EDB6ADF5050
:104A9000F36E010EDBCFF4FFF350F45C16E2010E6F
:104AA000DB50EA6A480FE96E040EEA22EF50E66E28
:104AB000D3C1E9FFD4C1EAFFD32B000ED423E552C2
:104AC000E750EF6E010EDB2AE2D7000ED880D655F4
:104AD000000ED75527E2BAC1E9FFBBC1EAFFEE528B
:104AE000080EEF6EBAC1E9FFBBC1EAFF020EE9266C
:104AF000000EEA22480EEE6E040EED6EB8C1E9FF1C
:104B0000B9C1EAFFEF50400B06E1BAC1E9FFBBC1F2
:104B1000EAFFC80E05D0BAC1E9FFBBC1EAFF880EA3
:104B2000EF6E25D0BAC1E9FFBBC1EAFFEE52080E15
:104B3000EF6EBAC1E9FFBBC1EAFF020EE926000E23
:104B4000EA22400EEE6E040EED6EBAC1E9FFBBC163
:104B5000EAFF840EEF6ED851D91107E005D0D9C114
:104B6000FAFF0101D851F96EFADF0101D59F020E5B
:104B7000E15C02E2E16AE552E16EE552E7CFD9FF7E
:104B80001200D9CFE6FFE1CFD9FFE6520101D08F65
:104B9000030EE66EE66AE66A710EE66E0F0EE66ECC
:104BA00067EC2CF0146E050EE15E1450DF6ADF50E6
:104BB000146E156A100E145C000E155810E2DF50CA
:104BC000040DF3CFE9FFF4CFEAFF000EE926040E4F
:104BD000EA22EE6AEE6AEE6AEE6ADF2AE8D76D8CA8
:104BE000010EE66EE66AE66AB70EE66E010EE66E46
:104BF00067EC2CF0146E050EE15E14506D9C010103
:104C0000080EC46F040EC56F000EB86F040EB96FA6
:104C1000B8C1BAF1BB6F42C4B6F1B65102E1100E91
:104C200012D0010EE66EE66AB60EE66E010EE66E74
:104C3000010EE66EE66A5AEC1AF0146E060EE15E9C
:104C400014500101200EB56FE552E552E7CFD9FFB0
:104C50001200D9CFE6FFE1CFD9FF020EE126000E08
:104C6000DE6E040EDD6EFD0EDB50E824166EFE0EC9
:104C7000DB50040DF3501624040DF350146E156A26
:104C8000020E0F0B05E0D89015321432E806FBE156
:104C9000D89014361536D89014361536D9CFE9FF8A
:104CA000DACFEAFF1450EE261550ED22DECFE9FFF1
:104CB000DDCFEAFFEF9EFD0EDB500AE1FE0EEA6A51
:104CC000DB34FE0BEA36E96EBC0EE926010E09D094
:104CD000FE0EEA6ADB34FE0BEA36E96EC40EE92604
:104CE000010EEA22DECFEEFFDDCFEDFFDECFE9FFE2
:104CF000DDCFEAFFEF9CDECFE9FFDDCFEAFF040E58
:104D0000E926000EEA22EF8C020EE15C02E2E16A83
:104D1000E552E16EE552E7CFD9FF1200D9CFE6FFA9
:104D2000E1CFD9FF020EE126FE0EDB50156A700FAF
:104D3000146E0F0E152214C0DEFF15C0DDFFDECF8E
:104D4000E9FFDDCFEAFFFD0EDBCFEFFFDBA407D0ED
:104D5000E66AFE0EDBCFE6FF7CDFE552E552FD0E94
:104D6000DBA208D0010EE66EFE0EDBCFE6FF71DFA0
:104D7000E552E552020EE15C02E2E16AE552E16EC3
:104D8000E552E7CFD9FF1200D9CFE6FFE1CFD9FF37
:104D9000020EE126FE0EDB5020E1BAC1E9FFBBC1E5
:104DA000EAFFEE52080EEF6EBAC1E9FFBBC1EAFF9F
:104DB000020EE926000EEA22400EEE6E040EED6EA3
:104DC000BAC1E9FFBBC1EAFF8C0EEF6EC4C1E9FFB7
:104DD000C5C1EAFF840EEF6E3BD0FD0EDB50E82428
:104DE000166EFE0EDB50040DF3501624040DF3CFA7
:104DF00014F0F4CF15F0000E1426040E152214C082
:104E0000DEFF15C0DDFF840EDECFE9FFDDCFEAFF58
:104E1000E850EF12FD0EDB50E824166EFE0EDB505C
:104E2000040DF3501624010F040DF3CF14F0F4CF4A
:104E300015F0000E1426040E152214C0DEFF15C056
:104E4000DDFF840EDECFE9FFDDCFEAFFE850EF1291
:104E5000020EE15C02E2E16AE552E16EE552E7CF63
:104E6000D9FF1200D9CFE6FFE1CFD9FF020EE1262C
:104E7000FD0EDB500AE0FE0EEA6ADB34FE0BEA367A
:104E8000E96EC40EE926010E09D0FE0EEA6ADB3493
:104E9000FE0BEA36E96EBC0EE926010EEA22EECFE1
:104EA000DEFFEDCFDDFFD9CFE9FFDACFEAFFEE502D
:104EB000ED1003E1F36AF46A44D0DECFE9FFDDCF01
:104EC000EAFF020EE926000EEA22FB0EDBCFEEFF20
:104ED000FC0EDBCFEDFFDECFE9FFDDCFEAFFEE52C8
:104EE000FA0EDBCFEFFF400EDECFE9FFDDCFEAFFAA
:104EF000E850EF16880EDECFE9FFDDCFEAFFE8507D
:104F0000EF12FD0EDB500AE0FE0EEA6ADB34FE0B08
:104F1000EA36E96EC40EE926010E09D0FE0EEA6AF1
:104F2000DB34FE0BEA36E96EBC0EE926010EEA22FE
:104F3000EF74DECF14F0DDCF15F014C0F3FF15C011
:104F4000F4FF020EE15C02E2E16AE552E16EE55235
:104F5000E7CFD9FF1200D9CFE6FFE1CFD9FF6DA887
:104F60004ED0FE0EEA6ADB34FE0BEA36E96EC40E62
:104F7000E926010EEA22EE50EFCFEAFFE96E400E7D
:104F8000EE16EE6AEE6AEE6AFE0EEA6ADB34FE0B9D
:104F9000EA36E96EC40EE926010EEA22EE50EFCFA2
:104FA000EAFFE96EEE7CFE0EEA6ADB34FE0BEA36BF
:104FB000E96EC40EE926010EEA22EF74400E146E6B
:104FC000FE0EEA6ADB34FE0BEA36E96EC40EE92611
:104FD000010EEA22EE50EFCFEAFFE96E1450EF1611
:104FE000FE0EEA6ADB34FE0BEA36E96EC40EE926F1
:104FF000010EEA22EE50EFCFEAFFE96EEF7CE552B8
:10500000E7CFD9FF12006D6A696A0101B56B120022
:105010000101B55113E16D6A696A160E6F6E9F0E3C
:105020006B6E7B0E696ED08EA28AA08AF28E6DB6F0
:0E50300002D06D86FCD70101010EB56F120093
:02503E0004016B
:1050400040511F0B010801E012004051600BE84283
:10505000E842E842E842E842010801E01200445117
:1050600003E0440501E012004151220A33E0030A43
:1050700026E0010A15E0210A0DE0010A01E0120014
:105080000101B30ECE6F020ECF6F080ED16FD26B3F
:10509000D08123D00101B30ECE6F020ECF6F1DD091
:1050A00046C4D6F147C4D7F10101000ED36F050EF7
:1050B000D46FBC0ED86F180ED96FD58F12000101B6
:1050C000880ECE6F050ECF6F070ED16FD26BC10E5B
:1050D000D06F120042C4AEF20101D08F1200050160
:1050E000886B4B0E896F8A6B8B6B8C6B8D6B080E8C
:1050F0008E6F0201A36BA26B1A0EE66E020EE66EB5
:105100008EEC26F0E552E5521E0EE66E030EE66EBC
:105110008EEC26F0E552E552400EE66E080EE66E85
:10512000050EE66EE66A030EE66E32EC27F0146EAC
:10513000050EE15E1450F3CFAAF2F4CFABF20201F8
:10514000AC6BAD6B1200D9CFE6FFE1CFD9FF020106
:10515000A26BAA51AB1102E1000E08D0AAC2E9FF6E
:10516000ABC2EAFFEF50800B01E0010E000945E100
:10517000FC0EDBCF14F0AAC2E9FFABC2EAFFEE528D
:10518000EF50D880145408E2AAC2E9FFABC2EAFF8C
:10519000EE52FC0EEFCFDBFFA26BFC0EDB50A25DEC
:1051A00019E2A251EA6A080FE96E050EEA22EF50F1
:1051B000E66EA251E76EFD0EDBCFE9FFFE0EDBCF00
:1051C000EAFFE750E926000EEA22E552E750EF6ECB
:1051D000A22BE3D7400EE66E080EE66E050EE66ED5
:1051E000E66A030EE66E32EC27F0146E050EE15E01
:1051F0001450F3CFAAF2F4CFABF20201A251E55260
:10520000E7CFD9FF1200D9CFE6FFE1CFD9FFA09AAF
:105210000201A3510CE1FD0EDBCFA4F2FE0EDBCFA9
:10522000A5F2FC0EDBCFA8F2010EA96FA36FA08A36
:10523000E552E7CFD9FF1200D9CFE6FFE1CFD9FF82
:10524000030EE126A09A0201A3512DE1DF6AFD0EB3
:10525000DBCF08F0FE0EDBCF09F0DE5208C0DEFF28
:1052600009C0DDFFDD52DF2ADF50146E156AFF0E24
:10527000141802E115500BE0010EDBCFE9FFDB2A29
:10528000020EDBCFEAFF01E3DB2AEF50ECE1FD0E7B
:10529000DBCFA4F2FE0EDBCFA5F2DFCFA8F2020136
:1052A000010EA96FA36FA08A030EE15C02E2E16A1E
:1052B000E552E16EE552E7CFD9FF1200D9CFE6FF04
:1052C000E1CFD9FF030EE126A09A0201A3512EE1FE
:1052D000DF6AFD0EDBCF08F0FE0EDBCF09F0DE52F9
:1052E00008C0DEFF09C0DDFFDD52DF2ADF50146E8B
:1052F000156AFF0E141802E115500CE0010EDBCF09
:10530000F6FFDB2A020EDBCFF7FF01E3DB2A080002
:10531000F550EBE1FD0EDBCFA4F2FE0EDBCFA5F2E4
:10532000DFCFA8F20201A96B010EA36FA08A030EC2
:10533000E15C02E2E16AE552E16EE552E7CFD9FFB6
:105340001200D9CFE6FFE1CFD9FF020EE126A09AE5
:105350000201AC51AD1102E1000E08D0ACC2E9FF70
:10536000ADC2EAFFEF50800B01E0010E000906E13B
:10537000030EA35D01E1A36BA35102E1A08A7ED0DD
:10538000020EA35D16E1E66A000EE66EE66A010E05
:10539000E66E030EE66E32EC27F0146E050EE15E4B
:1053A0001450F3CFACF2F4CFADF20201030EA36FB1
:1053B00064D0A30562E1400E146E156AA851145C16
:1053C000000E155803E2400EDF6E02D0A8C2DFFFC8
:1053D000DF50A85DA86F480EA66F050EA76F010EDF
:1053E000DFCFDBFFA95116E1010EDB5028E0A4C29C
:1053F000F6FFA5C2F7FF0800F550A6C2E9FFA7C255
:10540000EAFFEF6EA62B000EA723A42BA523010E07
:10541000DB06EAD7010EDB5012E0A4C2E9FFA5C209
:10542000EAFFEF50A6C2E9FFA7C2EAFFEF6EA62B84
:10543000000EA723A42BA523010EDB06EBD7020148
:10544000A85107E1400EDF5C02E1020E01D0030E1D
:10545000A36FDFCFE6FF480EE66E050EE66E010E87
:10546000E66E030EE66E32EC27F0146E050EE15E7A
:105470001450F3CFACF2F4CFADF2A08A020EE15C8F
:1054800002E2E16AE552E16EE552E7CFD9FF120090
:10549000006A0EAE4EEF2AF00E6C001E09AE53EFFE
:1054A0002AF0096C001EA5EC2CF009BE5DEF2AF075
:1054B00000AE000C096C056C000C00BE5AEF2AF01F
:1054C0000188FF0C006A0EAE6BEF2AF00D6C0E1E09
:1054D000E86A0E22001E09AE73EF2AF0086C091E5E
:1054E000E86A0922001E81EC2CF009BE83EF2AF045
:1054F00000AE000C086C091EE86A0922046C051E47
:10550000E86A0522000C00BE7AEF2AF00188FF0C41
:10551000006A0EAE93EF2AF00C6C0D1E0E1EE86AA8
:105520000D220E22001E09AE9DEF2AF0076C081E08
:10553000091EE86A08220922001E2DEC2CF009BE83
:10554000B0EF2AF000AE000C076C081E091EE86AD6
:1055500008220922036C041E051E04220522000CE9
:1055600000BEA4EF2AF00188FF0C09C013F008C0A8
:1055700012F008500D02F4CF07F0F3CF06F00950F7
:105580000E02F4CF09F0F3CF08F00D02F350072616
:10559000F4500822E86A092212500E02F35007263E
:1055A000F4500822E86A09220EAEDBEF2AF012500E
:1055B000085E1350095A13AE000C0D50085E0E50D1
:1055C000095A000C08C012F008500D02F4CF07F081
:1055D000F3CF06F009500E02F4CF09F0F3CF08F034
:1055E0000D02F3500726F4500822E86A09221250EF
:1055F0000E02F3500726F4500822E86A0922000C34
:1056000009C013F008C012F007C011F007500C02D7
:10561000F4CF05F0F3CF04F008500D02F4CF07F0FB
:10562000F3CF06F00C02F3500526F4500622E86A88
:10563000072211500D02F3500526F4500622E86AA5
:10564000072209500C02F3500626F4500722095095
:105650000D02086AE86A0822F3500726F45008226F
:1056600011500E02F3500626F4500722096AE86A28
:105670000822092212500E02F3500726F450082285
:10568000E86A092213500E02F3500826F45009224A
:02569000000C0C
:0E5692001201000202000008D804B2FB010061
:1056A0000102030109024300020100C028090400AD
:1056B0000001020201000524001001042402020579
:1056C00024060001052401000107058203080002E9
:1056D00009040100020A000000070503024000005F
:1056E00007058302400000040309043403410073EA
:1056F00000740072006F00670065006E0065003185
:10570000003000300030005F0073007400750066E8
:1057100000660000000000000000000000000034EF
:1057200003550053004200200053007400650070D0
:1057300000700065007200200046006F0063007575
:105740000073002000760030002E0031007300202E
:1057500000200016033000300030003000300030F0
:10576000003000300050003200A456E756EB561FC0
:0357700057535735
:0C5774002A0EF66E100EF76E000EF86E96
:1057800001010900F550F06F0900F550F16F03E1D8
:10579000F06701D03DD00900F550EB6F0900F550DE
:1057A000EC6F0900F550ED6F09000900F550E96E46
:1057B0000900F550EA6E090009000900F550EE6F86
:1057C0000900F550EF6F09000900F6CFF2F1F7CFAD
:1057D000F3F1F8CFF4F1EBC1F6FFECC1F7FFEDC147
:1057E000F8FF0101EE5302E1EF5307E00900F55025
:1057F000EE6EEE07F8E2EF07F9D7F2C1F6FFF3C15C
:10580000F7FFF4C1F8FF0101F007000EF15BBFD70D
:02581000120084
:0E581200056A046A036A026A200EE76ED890E7
:10582000063607360836093602360336043605369C
:105830000B50025C0C5003580D5004580E50055884
:1058400009E30B50025E0C50035A0D50045A0E50DF
:0A585000055A062AE72EE4D71200DD
:06585A00056A046A036AFE
:10586000180EE76ED8900736083609360336043628
:1058700005360C50035C0D5004580E50055807E3D4
:105880000C50035E0D50045A0E50055A072AE72E9D
:04589000EAD7120041
:0C589400D9CFE6FFE1CFD9FF020EE126DC
:1058A000040EDF6EDE52F40EDD6E010EDB06FDE14E
:1058B000DF06F8E1FE0EDB06F3E1020EE15C02E238
:0E58C000E16AE552E16EE552E7CFD9FF120032
:0258CE00FE0ECC
:1058D000E3CFE9FFFF0EE3CFEAFFE9CFF3FFEACF23
:1058E000F4FFFB0EE35003E1FC0EE35009E0FB0E76
:1058F000E30602E2FC0EE306FD0EE350EE6EF1D786
:02590000120093
:0E590200056A046A100EE76ED8900836093662
:10591000043605360D50045C0E50055805E30D5055
:0E592000045E0E50055A082AE72EF0D712003A
:02592E0013EE76
:1059300000F023EE00F0F86A019CBAEC2BF0C7EC03
:0A5940002CF080EC09F0FBD71200F8
:06594A00056A080EE76E7D
:10595000D890093605360E50055C02E3056E092A1B
:06596000E72EF7D712004C
:0A5966000101020304050607080909
:105970000A0B0C0F1114191E2531496394B9D2F981
:0E59800000EE00F00F0EEE6AEA62FDD7120094
:02598E00120005
:105990000000000A00000000002D39393900000025
:1059A00000000000000001000000000000000003F3
:1059B00000000000000100020401080000000002D5
:1059C0000604050109080A0605090A00000000028C
:1059D0000104080000000002030105040C080A038A
:1059E000050C0A000000000201080400000000028B
:1059F000030109080C040603090C0600000000005E
:105A000003080F1013181B2027282B3033383F4072
:105A10004300000000000000000000000000000043
:105A20000000000000000000000000000000000076
:025A3000000074
:020000040030CA
:0100000024DB
:010001000EF0
:0100020036C7
:010003001EDE
:010005008179
:010006008178
:010008000FE8
:01000900C036
:01000A000FE6
:01000B00A054
:01000C000FE4
:01000D0040B2
:00000001FF
